:10E00000B240805A20013F4002000F9305242F8325
:10E010009F4FBAE80002FB233F4003000F93042404
:10E020001F83CF430202FC233040D4E2304030E073
:10E03000001332C2D24276000402A2D3020232D2CC
:10E0400000130F1232C2E2B32300022492D3020261
:10E05000C243230032D23F4100130E430E9F132CC4
:10E060000343034303430343034303430343034380
:10E070000343034303430343034303430343034370
:10E080001E530E9FED2B30410B120A12091208127B
:10E09000084E094FB012FAE00A4E0B4FB012FAE0E8
:10E0A0000A9EF8230B9FF623F2D0E0FF5600B01231
:10E0B000FAE00A4E0B4F5F42560012C34F104F1149
:10E0C0004F114F114F114E4F0F430C480D490C8A01
:10E0D0000D7B0E2C3E533F634E5E4E5E4E5E4E5E9B
:10E0E0004E5EC24E56003F401000B0125AE0DF3F75
:10E0F000384139413A413B4130410B120A1232C298
:10E10000B2400002600192C3600182437001B240DC
:10E1100000516601B2D02000600192B36601FD2774
:10E1200092C366011E42760192B36601FD2792C337
:10E1300066011F427601B2F0EFFF600132D20F8E0E
:10E140000A4F3C40FA0F0B430A9301343B430D4303
:10E150000C9301343D43B0128AE83A413B413041CF
:10E16000B240805A2001F24005002100C24329003C
:10E17000F2421900C2432600C2432E00F240300092
:10E180001B00F240F9FF2200F2432A00F240DBFFBD
:10E190001A00E2432400C2432C00E2432500C2439C
:10E1A0002D00F240B7FF5700F2D0E0FF5600D243F7
:10E1B00058003041F2D030001B00D2D37000D2C3DF
:10E1C0000500F2D003000500F24011007000F2409B
:10E1D00020007100F24040007400C2437500C24349
:10E1E0007300D2C37000D2D3010030414E4FE2B36E
:10E1F0000300FD27C24E770030410B120A120912AC
:10E20000094F4A4E4B434B9E082C4F4B0F596F4FB3
:10E21000B012ECE15B534B9AF82B39413A413B4148
:10E2200030411B5B33326D283131352E322D382D84
:10E230003120584F4E2F584F464629204543484FCE
:10E24000204F46460D0A0047696E67657220546587
:10E25000726D696E616C2052656164790D0A1B5B99
:10E2600033306D0050434C007265626F6F74007202
:10E270006563616C00474E443A50434C20526563DD
:10E28000616C0D0A00474E443A50434C205265637E
:10E29000616C2064756520746F2064726966740D0A
:10E2A0000A0066726571006563686F206F6E0045D5
:10E2B00063686F206973204F4E0D0A006563686FB5
:10E2C000206F6666004563686F206973204F46467D
:10E2D0000D0A0000314068028143900081439200A2
:10E2E0008143940081439600B01260E1F2C21900AC
:10E2F000B012B4E13F40FF00B0125AE03F43B01209
:10E300005AE0F2D219003E40C8803F407000B0127F
:10E3100088E03F43B0125AE0B012FAE0064E074FD1
:10E320000C4E0D4F3A4000C21B43B0128EE8054C14
:10E330000C460D473A4000C21B43B0128EE80A4E0D
:10E340000B4F3C40FF000D43B0126AE80C4E0D4FDE
:10E350003A4000C21B43B0128EE8C2457400C24C62
:10E3600073007F400D00B012ECE17F400A00B01254
:10E37000ECE17E4024003F4022E2B012FAE17E4010
:10E380001C003F4047E2B012FAE182430202C2435E
:10E390002B00C243230032D2044392B302021F2453
:10E3A00032C214433F4040000F51B01220E64C4FA0
:10E3B0008C11E2C3230092C302020F410F5CFF40A5
:10E3C0000D003F000F4C0F51FF400A0040001C534E
:10E3D0004E4C3F4040000F51B012FAE132D2A2B28F
:10E3E0000202502432C21443A2C202023D40030082
:10E3F0000E413F4064E2B012BCE70F9303213E4060
:10E4000068E20F41B012ECE70F93F8203E406FE254
:10E410000F41B012ECE70F93C7243E40C8803F4045
:10E420007000B01288E03F43B0125AE0B012FAE038
:10E43000064E074F0C4E0D4F3A4000C21B43B01220
:10E440008EE8054C0C460D473A4000C21B43B01203
:10E450008EE84FEE0FEE8F107EF38E100C4E0D4FA8
:10E460003A4000C21B43B0128EE8C2457400C24C51
:10E4700073007E400F003F4075E2B012FAE1814325
:10E48000900032D2A2B302021E2432C21443A2C3AD
:10E4900002025E4204027E9275247E900D000724E3
:10E4A0001F4190000F51CF4E000091539000B1904A
:10E4B0003D009000642CF2900D0004025D249193C5
:10E4C0009200552432D20493672332C291539400B0
:10E4D000816396001E4194001F4196003E80818416
:10E4E0003F701E0042288143940081439600B01281
:10E4F000FAE00E860F773E50204E0F633E80419C1F
:10E500000F7333283E40C8803F407000B01288E04F
:10E510003F40FF00B0125AE0B012FAE0064E074F3B
:10E520000C4E0D4F3A4000C21B43B0128EE8054C12
:10E530000C460D473A4000C21B43B0128EE84FEE26
:10E540000FEE8F107EF38E100C4E0D4F3A4000C22E
:10E550001B43B0128EE8C2457400C24C73007E406B
:10E560001C003F4085E2B012FAE132D2153F5F4213
:10E570000402B012ECE1A63F81939000A027A2D242
:10E5800002029D3F1F4190000F51CF430000819335
:10E5900090000224B15390007F42B012ECE17F4022
:10E5A0002000B012ECE1833F3E40A2E20F41B012E6
:10E5B000ECE70F930324B012FAE0613F3E40A7E27C
:10E5C0000F41B012ECE70F9309247E400C003F404E
:10E5D000AFE2B012FAE191439200513F3E40BCE2FB
:10E5E0000F41B012ECE70F934A277E400D003F40E9
:10E5F000C5E2B012FAE181439200413FB240085AAD
:10E600002001FF3F5F4190005F534E4F0F41B0121A
:10E61000E4E6E2C32300333F315098003040B8E8CD
:10E620000B120A120912094F4D430B430C43E2C26D
:10E630002200E2B320000B241B530C633B9020A16B
:10E6400003203C9007003F24E2B32000F523D2C30F
:10E650002100B240085A20013E424D5DE2B2200046
:10E66000FD23E2B320004F434F634DDFD2D321009F
:10E67000E2B22000FD27D2C321003E53EE234A4DD3
:10E680000C430B4A3B530C9B222CB240085A2001EE
:10E690003E424D5DE2B22000FD23E2B320004F4335
:10E6A0004F634DDFD2D32100E2B22000FD27D2C359
:10E6B00021003E53EE230F490F5CCF4D00001C5349
:10E6C0000C9BE32B043CB240085A2001FF3FD2D3FD
:10E6D0002100B240805A20014F4A8F1139413A41FE
:10E6E0003B4130410B120A120A4F0C430D43E2B377
:10E6F000200002200F435F3CE2D22200D2C321005F
:10E70000E2B320000B241C530D633C9020A1032096
:10E710003D9007004C24E2B32000F523B240085A94
:10E7200020014D4E3C42E2B32000FD234F4D4F5F90
:10E730004F434F6FC2DF2100E2C22100E2B320004D
:10E74000FD27E2D22100D2C321004D5D3C53EB23D3
:10E750004B4E0E431B932124B240085A20010F4A0E
:10E760000F5E6D4F3C42E2B32000FD234F4D4F5FE3
:10E770004F434F6FC2DF2100E2C22100E2B320000D
:10E78000FD27E2D22100D2C321004D5D3C53EB2393
:10E790001E530F4B3F530E9FDF2BE2C22200F2D0DD
:10E7A00005002100B240805A20011F43043CB240C2
:10E7B000085A2001B03F3A413B4130410B120B4D0A
:10E7C0000D930A240C4F0D4E6E4D1D536F4C1C5370
:10E7D0004F9E04203B53F8230C43053C5C4CFFFF49
:10E7E0005F4DFFFF0C8F0F4C3B4130410B120A1263
:10E7F000091208120B4F0A4E694E1A5349931524F9
:10E80000084A18831853C8930000FC23088A6F4BEA
:10E810001B534F930C244F99FA230D480E4A0F4B6C
:10E82000B0123AE80F93F3233B530F4B013C0F43D5
:10E83000384139413A413B4130410B120B4F0D9366
:10E8400002200D430F3C6F4E1E536C4B4C9F062015
:10E850001B534C93F6273D53F623F33F4D4C5F4E2D
:10E86000FFFF0D8F0F4D3B4130410E430F43083CDE
:10E8700012C30D100C1002280E5A0F6B0A5A0B6BA4
:10E880000C93F6230D93F423304130406AE80FEFE8
:10E890000EEE394021000A3C08100E6E0F6F0F9BE0
:10E8A000052802200E9A02280E8A0F7B0C6C0D6D33
:0AE8B00008681983F1233041FF3F8F
:02E8BA0000005C
:10FFE0002CE02CE042E02CE02CE02CE02CE032E095
:10FFF0002CE02CE02CE02CE02CE02CE02CE000E0CD
:040000030000E00019
:00000001FF
